S0220000687474703A2F2F737265636F72642E736F75726365666F7267652E6E65742F1D
S12300000C9438000C9461150C94DF1B0C945F000C945F000C945F000C945F000C945F0059
S12300200C945F000C949B1C0C945F000C948C200C945F000C943A160C9414160C940215AB
S12300400C94C0210C945F000C940B210C945F000C946C220C9434220C945F000C945F002F
S12300600C945F000C945F000C945F000C945F0011241FBECFEFD0E1DEBFCDBF14BEA895C7
S123008088E10FB6F89480936000109260000FBE15E0A0E0B1E0E2E5F8E402C005900D92C1
S12300A0AA31B107D9F716E0AAE1B5E001C01D92A03BB107E1F70E94950D0C9428240C9418
S12300C0000020E030E0D901AC54BF4F0E940A24802DF901EF5BFE4F80832F5F3F4F203A9D
S12300E0310589F720E030E0D901A857BE4F0E940A24802DF901E65CFE4F80832F5F3F4F2B
S12301002530310589F712BC11BC089520E030E0F901EF5BFE4F8081D901AC54BF4F082ED8
S12301200E9417242F5F3F4F203A310589F712BC11BC08954E9B11C020E030E0D9015096F0
S12301400E940A24802DF901EF51FE4F80832F5F3F4F203A310591F0F1CF20E030E0D901BD
S1230160A859BD4F0E940A24802DF901EF51FE4F80832F5F3F4F203A310589F712BC11BCA0
S123018008954E9B11C020E030E0F901EF51FE4F8081D9015096082E0E9417242F5F3F4F7D
S12301A0203A310591F0F1CF20E030E0F901EF51FE4F8081D901A859BD4F082E0E941724D8
S12301C02F5F3F4F203A310589F712BC11BC089520E931E0D9010E940A24802D2055314060
S12301E0F901EF57FD4F80832F5A3E4F81E0203F380781F712BC11BC089520E430E0F90199
S1230200EF57FD4F8081D901A05BBE4F082E0E9417242F5F3F4F203A310589F712BC11BC8B
S12302200895A2E0B0E00E940A24802D90E090931D0180931C0120911C0130911D01A3E07D
S1230240B0E00E940A24802D90E0982F8827820F931F90931D0180931C01ADEEB3E00E9423
S12302600A24802D90E090932101809320012091200130912101AEEEB3E00E940A24802D55
S123028090E0982F8827820F931F909321018093200180911C0190911D0190931F018093F5
S12302A01E01A4E0B0E00E940A24802D90E090932301809322012091220130912301A5E05F
S12302C0B0E00E940A24802D90E0982F8827820F931F9093230180932201A6E0B0E00E94AF
S12302E00A24802D90E090930101809300012091000130910101A7E0B0E00E940A24802D6D
S123030090E0982F8827820F931F9093010180930001A1E0B0E00E940A24802D80931A05B7
S1230320A8E0B0E00E940A24802D80931301A9E5B1E00E940A24802D80932C01A2E0B4E00B
S12303400E940A24902D892F8150843078F080912C01843039F481E08093180183E680933F
S1230360C00506C082E08093180102C090931801A9E0B0E00E940A24802D80931201AEE018
S1230380B0E00E940A24802D80932501ABE0B0E00E940A24802D80931901ACE0B0E00E9490
S12303A00A24802D80931A01AFE6B1E00E940A24802D80931B01A2EFB1E00E940A24802DBF
S12303C08093880580918805882319F081E080938805ADE0B0E00E940A24802D26E0829F65
S12303E0C00111249093150180931401A1E7B1E00E940A24802D8093E405A0E7B1E00E9456
S12304000A24802D8093E2058AE08093110681E080930F06AFE8B1E00E940A24802D80932E
S12304202D0180912D0181FF05C080912D01827F80932D0180912D0185FF05C080912D01BE
S12304408F7280932D01A4EFB1E00E940A24802D24E1829FC00111249093BB058093BA05E4
S1230460A5EFB1E00E940A24802D8093B705A6EFB1E00E940A24802D8093B505A7EFB1E070
S12304800E940A24802D8093B405A8EFB1E00E940A24802D90E09093B3058093B2052091A4
S12304A0B2053091B305A9EFB1E00E940A24802D90E0982F8827820F931F9093B30580934B
S12304C0B205ABEFB1E00E940A24802D90E090932F0180932E0120912E0130912F01ACEF48
S12304E0B1E00E940A24802D90E0982F8827820F931F90932F0180932E01ADEFB1E00E945D
S12305000A24802D90E090933101809330012091300130913101AEEFB1E00E940A24802D73
S123052090E0982F8827820F931F9093310180933001AFEFB1E00E940A24802D90E09093B6
S12305403301809332012091320130913301A0E0B2E00E940A24802D90E0982F8827820F3E
S1230560931F909333018093320120E030E0D901A25ABE4F0E940A24802DF901EF5DFC4F27
S12305808083D901AE58BE4F0E940A24802DF901EF53FA4F8083D901A458BE4F0E940A24AF
S12305A0802D808B2F5F3F4F2A30310501F7A7E0B2E00E940A24802D80933601A3E0B2E0E6
S12305C00E940A24802D8093370120E030E0F901E251FA4F84E6808BD901A45EBD4F0E94CA
S12305E00A24802D80832F5F3F4F2031310579F720E030E0D901A759BE4F0E940A24802D92
S1230600F901E95DFE4F80832F5F3F4F2430310589F720E030E0D901A25DBD4F0E940A245B
S1230620802DF901EF50FB4F80832F5F3F4F2031310589F7ADE6B1E00E940A24802D8093AC
S12306402401A1EFB1E00E940A24802D80938705A0EFB1E00E940A24802D80932B01A6E0D2
S1230660B2E00E940A24802D8093260120E030E0D901AA54BC4F0E940A24802DF901E55D81
S1230680FC4F80832F5F3F4F2031310589F7A7ECB3E00E940A24802D80933801A8ECB3E0CF
S12306A00E940A24802D8093390112BC11BC089580911C0190911D01A2E0B0E0082E0E94DD
S12306C0172480911C0190911D01892F9927A3E0B0E0082E0E941724809122019091230157
S12306E0A4E0B0E0082E0E9417248091220190912301892F9927A5E0B0E0082E0E941724B6
S12307008091000190910101A6E0B0E0082E0E9417248091000190910101892F9927A7E043
S1230720B0E0082E0E94172480911301A8E0B0E0082E0E94172480911201A9E0B0E0082E4F
S12307400E94172412BC11BC089580E0A1EFB1E0082E0E9417248AE0A0EFB1E0082E0E948A
S1230760172480918805A2EFB1E0082E0E94172484E0A9E5B1E0082E0E94172485E0ACE0E0
S1230780B0E0082E0E94172482E3AFE6B1E0082E0E94172424E1A1E7B1E0022E0E941724E9
S12307A091E0A0E7B1E0092E0E94172488ECA4EFB1E0082E0E941724A5EFB1E0092E0E94EF
S12307C01724A6EFB1E0022E0E9417248AE5A7EFB1E0082E0E94172488EEA8EFB1E0082E2A
S12307E00E94172483E0A9EFB1E0082E0E94172480912E0190912F01ABEFB1E0082E0E94E5
S1230800172480912E0190912F01892F9927ACEFB1E0082E0E9417248091300190913101BC
S1230820ADEFB1E0082E0E9417248091300190913101892F9927AEEFB1E0082E0E94172426
S12308408091320190913301AFEFB1E0082E0E9417248091320190913301892F9927A0E028
S1230860B2E0082E0E9417248CEDA7E0B2E0082E0E94172486EEA3E0B2E0082E0E9417248E
S12308802CE132E088ECD901082E0E9417242F5F3F4F82E02C323807A9F782E2AFE8B1E08D
S12308A0082E0E94172481E0A6E0B2E0082E0E94172412BC11BC0895CF92DF92EF92FF9279
S12308C00F931F93CF93DF93C0E0D0E0A5E0B2E00E940A24202D30E040E050E0A3EDB3E0E5
S12308E00E940A24602D6E01CC0CDD1C8BE393E0C80ED91EF601E080F18070E080E090E0C1
S12309000E947B2300E010E0A80197010E947B2324E630E040E050E00E94CD2379018A0141
S1230920CA01B90124EF31E040E050E00E947B2328EC30E040E050E0E20EF31E041F151FAE
S1230940A80197010E94CD23CA01B9012FEF30E040E050E00E947B2325E030E040E050E018
S12309600E94CD2382E0220F331F441F551F8A95D1F7CA01B90124E630E040E050E00E94AD
S1230980CD23F601318320832196C732D10509F09DCFC0E0D0E0A9ECB3E00E940A24202D95
S12309A030E040E050E0A3EDB3E00E940A24602D6E01CC0CDD1C89E893E0C80ED91EF6016B
S12309C0E080F18070E080E090E00E947B2300E010E0A80197010E947B2324E630E040E057
S12309E050E00E94CD2379018A01CA01B90124EF31E040E050E00E947B2328EC30E040E0AF
S1230A0050E0E20EF31E041F151FA80197010E94CD23CA01B9012FEF30E040E050E00E94D2
S1230A207B2325E030E040E050E00E94CD2312E0220F331F441F551F1A95D1F7CA01B901D5
S1230A4024E630E040E050E00E94CD23F601318320832196C732D10509F09DCFC0E0D0E00D
S1230A60AAECB3E00E940A24202D30E040E050E0A3EDB3E00E940A24602D6E01CC0CDD1C0C
S1230A8087ED93E0C80ED91EF601E080F18070E080E090E00E947B2300E010E0A801970165
S1230AA00E947B2324E630E040E050E00E94CD2379018A01CA01B90124EF31E040E050E0F8
S1230AC00E947B2328EC30E040E050E0E20EF31E041F151FA80197010E94CD23CA01B901AE
S1230AE02FEF30E040E050E00E947B2325E030E040E050E00E94CD23A2E0220F331F441FD5
S1230B00551FAA95D1F7CA01B90124E630E040E050E00E94CD23F601318320832196C732D7
S1230B20D10509F09DCFC0E0D0E0A4E0B2E00E940A24202D30E040E050E0A3EDB3E00E94CE
S1230B400A24602D6E01CC0CDD1C85E294E0C80ED91EF601E080F18070E080E090E00E9464
S1230B607B2300E010E0A80197010E947B2324E630E040E050E00E94CD2379018A01CA01B6
S1230B80B90124EF31E040E050E00E947B2328EC30E040E050E0E20EF31E041F151FA8016E
S1230BA097010E94CD23CA01B9012FEF30E040E050E00E947B2325E030E040E050E00E94BD
S1230BC0CD23E2E0220F331F441F551FEA95D1F7CA01B90124E630E040E050E00E94CD233D
S1230BE0F601318320832196C732D10509F09DCFDF91CF911F910F91FF90EF90DF90CF90BC
S1230C000895EAE7F0E0108210927C0010921B0580E880BF87EE808311B882E890E090933B
S1230C201D0580931C0584E690E090931F0580931E0590932B0580932A0508950F931F937D
S1230C40CF93DF93282F30E0F901EE0FFF1FEE5FFE4F0081118143E0033F140718F0E2E346
S1230C60F0E04CC053E00F3D150718F0EAE0F0E045C0C0E0D0E087E290E0A901489F900107
S1230C80499F300D589F300D1124D901AC0FBD1FAA0FBB1FA55CBC4F8D919C911197801728
S1230CA0910730F5FE013197E20FF31FEE0FFF1FE55CFC4F20813181608171814D915C9111
S1230CC0FE01EE0FFF1FEE0FFF1FEC0FFD1F3596201B310BC901880F991F880F991F641B9B
S1230CE0750B820F931F0E94A623E60FF71F06C02196C732D10549F6E8ECF0E0CF01DF9148
S1230D00CF911F910F9108950F931F93CF93DF93AC01E0E0F0E0EF01CC0FDD1FDE01AD5872
S1230D20BB4F8D919C91119748175907C0F56D917C913197EE0FFF1FDF01AD58BB4F8D9143
S1230D409C911197681B790B8D919C91C557DB4F28813981E557FB4F00811181481B590B5F
S1230D6084E690E0DC014A9FC0014B9F900D5A9F900D11240E94A623201B310B0190F081D8
S1230D80E02D629FC001639F900D729F900D112464E670E00E94A6236E0F7F1F09C031964E
S1230DA0EA30F10509F0B7CF60919F047091A004CB01DF91CF911F910F9108950F931F938A
S1230DC0CF93DF93AC018091B3049091B4044817590718F4E0EFF0E057C08091CF04909167
S1230DE0D0048417950718F4E0E0F0E04DC0E1E0F0E0EF01CC0FDD1FDE01AD54BB4F8D91DB
S1230E009C91119748175907C0F56D917C913197EE0FFF1FDF01AD54BB4F8D919C911197B9
S1230E20681B790B8D919C91EF52FB4F20813181CF52DB4F08811981481B590B84E690E06F
S1230E40DC014A9FC0014B9F900D5A9F900D11240E94A623201B310B0190F081E02D629FC3
S1230E60C001639F900D729F900D112464E670E00E94A623E61BF70B07C03196EE30F10581
S1230E8009F0B7CFEEEFF0E0CF01DF91CF911F910F910895A89582E50E94C12283E10E9466
S1230EA0C12280917B0590917C05892F99270E94C12280917B0590917C050E94C122809152
S1230EC03205909133050E94C12280912C0590912D050E94C12280911C0590911D050E94C8
S1230EE0C12280912A0590912B050E94C12280912805909129050E94C12280912405909188
S1230F0025050E94C12280918105909182056091180170E00E94A623CB010E94C1228091B8
S1230F2080050E94C12280917F050E94C1222091EC053091ED058091BC059091BD05E3E0BC
S1230F4096958795EA95E1F78170232F3327822B0E94C1228091EC059091ED050E94C12286
S1230F608091B6050E94C12280910E060E94C12280912205909123050E94C1228091BE0598
S1230F809091BF05969587950E94C1228091810090E0909337058093360589B1869586957D
S1230FA0817090E0909339058093380583B18695817090E090933B0580933A05209193056D
S1230FC030E0220F331FF901E45DFA4F80819181892F990F990B93E0220F331F9A95E1F7E2
S1230FE0822B0E94C122E0919305F0E0EE0FFF1FE45DFA4F808191810E94C1228DEA0E948C
S1231000C122809193058F5F80939305883010F0109293050895CF92DF92EF92FF920F9392
S12310201F93CF93DF93A89588E10FB6F89480936000109260000FBE0E940D23882309F473
S12310406AC50E949E2290939205809391058236910509F4E8C28336910508F041C08035A6
S1231060910509F45AC381359105E8F48534910509F4D1C08634910568F48932910509F4BD
S12310809DC48134910509F48DC08832910509F040C571C48634910509F446C18D34910528
S12310A009F037C5BDC18535910509F4EAC38635910548F48235910509F4ABC3833591052C
S12310C009F027C5CDC48835910509F422C48136910509F442C08735910509F01AC594C393
S12310E08936910509F4CAC28A369105C8F48536910509F408C28636910548F48336910507
S123110009F494C28436910509F003C504C58636910509F4E7C08736910509F0FAC4D5C207
S12311208037910509F4FEC28137910548F48D36910509F434C18F36910509F0EAC401C405
S12311408937910509F45DC48A37910509F471C28837910509F0DDC46CC281E60E94C12287
S123116080EA0E94C12210929205109291050EC0EF5BFE4F80810E94C12280919105909158
S1231180920501969093920580939105E0919105F0919205E03AF10558F382E30E94122205
S12311A08EE9B7C41092920510929105C0E0D0E00E940D23882341F1C0919105D0919205EA
S12311C0C03AD10589F40E949E2290939205809391058E3B910519F4C6E1DAEF15C0809137
S12311E091050E94C122FBCF0E949E22CF5BDE4F8883809191059091920501969093920592
S123120080939105C0E0D0E021964AEFC030D40708F081C4CDCFC0E0D0E00E940D23882370
S123122009F459C00E949E228A3B910509F073C488E10FB6F89480936000109260000FBEAB
S123124010929205109291053EC0885B0E94C1228DEF0E94C12220919105309192058AEF9A
S123126090E0289FE001299FD00D389FD00D112407C0DE010E940A24802D0E94C122219665
S123128020919105309192052F5F3F4F8AEF90E0AC01249FC001259F900D349F900D11246F
S12312A021503040C817D90720F3822F885B80950E94C12280919105909192050196909330
S12312C092058093910580919105909192058430910508F4BACF21965AEFC030D50708F0D8
S12312E01AC49BCF86E60E94C12280EA0E94C12210929205109291050EC0EF51FE4F8081F5
S12313000E94C122809191059091920501969093920580939105E0919105F0919205E03AB2
S1231320F10558F389E9F5C3109292051092910500E010E00E940D23882349F1C09191055F
S1231340D0919205C03AD10591F40E949E229093920580939105893B910519F406E11AEF20
S123136016C0E0918F05F0919005099510C00E949E22CF51DE4F88838091910590919205F1
S12313800196909392058093910500E010E00F5F1F4F8AEF0030180708F0BDC3CBCF8DE656
S12313A00E94C12289E00E94C12280911C0190911D010E94C12280911C0190911D01892F9F
S12313C099270E94C12280912201909123010E94C1228091220190912301892F99270E9433
S12313E0C12280910001909101010E94C1228091000190910101892F99270E94C122809109
S123140013010E94C122809112010E94C122AAE0B0E00E940A24802D0E94C12282E979C3C3
S12314201092920510929105C0E0D0E00E940D238A3008F461C00E949E2290931D01809388
S12314401C0100911C0110911D010E949E22982F8827800F911F90931D0180931C010E94D4
S12314609E22909323018093220100912201109123010E949E22982F8827800F911F909378
S12314802301809322010E949E22909301018093000100910001109101010E949E22982FF5
S12314A08827800F911F90930101809300010E949E22809313010E949E22809312010E944E
S12314C09E22AAE0B0E0082E0E9417240E94501C0E949E22823B910551F40E945803E091A5
S12314E08F05F09190050995CFE6DAEF05C0E0918F05F0919005099521964AEFC030D407E9
S123150008F009C393CF85E60E94C12283E10E94C12210929205109291050EC0EF5DFC4FF2
S123152080810E94C122809191059091920501969093920580939105E0919105F0919205A9
S1231540EA30F10558F3809119010E94C12280911A010E94C12283E00E9413228091270158
S12315600E94C122809128010E94C122809129010E94C12280912A010E94C122809114017C
S12315809091150166E070E00E94A623CB010E94C122809124010E94C122AEE6B1E00E943C
S12315A00A24802D0E94C1228AE90E94C1228CE60E94C12284E10E94C12210929205109213
S12315C091050EC0EF53FA4F80810E94C12280919105909192050196909392058093910539
S12315E0E0919105F0919205EA30F10558F310929205109291050EC0EF53FA4F80890E94F8
S1231600C122809191059091920501969093920580939105E0919105F0919205EA30F1055B
S123162058F383E976C20E94860075C20E94C10072C20E944A076FC20E949E22C82FD0E094
S12316400E949E22C817D90709F065C20E949E228C0190939205809391050E949E22081772
S1231660190709F058C20E949E228639910509F052C280919105CF5BDE4F4DC00E940D2392
S12316808530D0F6FBCF0E949E22C82FD0E00E949E22C817D90709F03EC20E949E228C01EF
S12316A090939205809391050E949E220817190709F031C20E949E228839910509F02BC297
S12316C080919105CF51DE4F26C00E940D238530D0F6FBCF0E949E22C82FD0E00E949E22AA
S12316E0C817D90709F017C20E949E228C0190939205809391050E949E220817190709F069
S12317000AC20E949E228F3A910509F004C280919105CF57DD4F8883FEC10E940D2385302F
S1231720C8F6FBCFC0E0D0E00E940D23823080F10E949E220E949E228F38910509F0EBC112
S123174010929205109291051CC0EF57FD4F108180E70E94C12282E00E94C122809191059B
S12317600E94C122812F0E94C1228FE80E94C12280919105909192050196909392058093EC
S12317809105E0919105F0919205E03AF105E8F221965AEFC030D50709F4BDC1C5CF0E9429
S12317A09E228C010E949E22F82EEE24E00EF11E0E949E228C0190939205809391050E944D
S12317C09E220817190709F0A6C10E949E22883A9105A9F4D7010E941224E07080919105A8
S12317E090919205E82BF92BF0939205E0939105D7010F010E94232412BC11BC8CC1E091A9
S12318008F05F091900509950E940D23853038F6FBCFCC24DD240E940D23833040F10E94B4
S12318209E22EC010E949E228C010E949E228D3A910509F070C1102F00270C0F1D1FD80189
S12318400E940A24F02C84E50E94C12283E00E94C1228F2D0E94C122802F0E94C122012F1D
S12318601127802F0E94C1228BEA0E94C1220894C11CD11C80E0C8168AEFD80609F44BC1FA
S1231880CACFCC24DD240E940D238330C0F10E949E22EC010E949E227C010E949E228A3A30
S12318A0910509F038C1FE2CEE24EC0EFD1ED7010E940A24802D90E0D70111960E940A2437
S12318C0002D10E0102F0027080F191F85E50E94C12284E00E94C122802F0E94C122012FF6
S12318E01127802F0E94C1228E2D0E94C122EF2CFF248E2D0E94C1228AEA0E94C122089425
S1231900C11CD11C40E0C4164AEFD40609F403C1BACFC0E0D0E00E940D23882359F00E94EA
S12319209E22873A910509F0F6C0E0918F05F0919005099521965AEFC030D50709F4EBC0B0
S1231940EACFC0E0D0E00E940D23882369F00E949E228039910509F0DEC00E94FD00E0914C
S12319608F05F0919005099521968AEFC030D80709F4D1C0E8CFC0E0D0E00E940D2388230A
S1231980B1F00E949E22873D910509F0C4C08091280590912905ADE6B1E0082E0E941724A5
S12319A012BC11BCE0918F05F0919005099521964AEFC030D40709F4AEC0DFCFC0E0D0E0AB
S12319C00E940D238823B1F00E949E22863D910509F0A1C08091280590912905AEE6B1E01E
S12319E0082E0E94172412BC11BCE0918F05F0919005099521965AEFC030D50709F48BC068
S1231A00DFCFC0E0D0E00E940D23823010F10E949E22892B09F07FC00E949E22863891053B
S1231A20C1F489E70E94C12285E00E94C1228FEC0E94C1228FE30E94C1228CE00E94C12226
S1231A408EE00E94C1228BE00E94C12286E80E94C12221968AEFC030D80709F45CC0D3CFF2
S1231A60C0E0D0E00E940D23823008F44CC00E949E22892B09F047C00E949E228C3A9105B2
S1231A8009F049C083E50E94C12288E00E94C1228091B0059091B1050E94C1228091B0057E
S1231AA09091B105892F99270E94C1228091EA059091EB050E94C1228091EA059091EB05A7
S1231AC0892F99270E94C1228091E5059091E6050E94C1228091E5059091E605892F9927FA
S1231AE00E94C12280911806909119060E94C1228091180690911906892F99270E94C122FD
S1231B008CEA0E94C12221964AEFC030D40719F0A9CF0E94C122A895DF91CF911F910F91A8
S1231B20FF90EF90DF90CF9008950F931F93CF93DF931092ED051092EC050E940A223C9A35
S1231B403D9A3F9A3E9A449A449A479A469A38984098399841983A9842983B984398389800
S1231B6039983A983B9854985C9855985D9854985598239A249A259A2B9A2C982D98279A07
S1231B80269A5398529822985698219820980E941522AAE5B1E00E940A24802D809389057C
S1231BA00E94051C0E94501C0E94F8210E9401060E945C042B9A2C98A7E0B0E00E940A247A
S1231BC0802D12BC11BC85FF9BC080910001909101019F7D90930101809300010E94580353
S1231BE00E94A5030E94C1000E9486000E94FD0086E0AAE0B0E0082E0E94172489E1ABE0E5
S1231C00B0E0082E0E9417248EE1ACE0B0E0082E0E941724AEE0B0E0082E0E94172420E04E
S1231C2030E0F901EF5DFC4F8081D901A25ABE4F082E0E9417242F5F3F4F2A30310589F7DC
S1231C4080912701A9E6B1E0082E0E94172480912801AAE6B1E0082E0E941724809129016B
S1231C60ABE6B1E0082E0E94172480912A01ACE6B1E0082E0E94172420E030E0F901EF536D
S1231C80FA4F8081D901AE58BE4F082E0E9417242F5F3F4F2A30310589F720E030E0F901C0
S1231CA0EF53FA4F8089D901A458BE4F082E0E9417242F5F3F4F2A30310589F78091E40570
S1231CC0A1E7B1E0082E0E941724809114019091150166E070E00E94A623ADE0B0E0062E25
S1231CE00E94172484E1ADE6B1E0082E0E94172481EEAEE6B1E0082E0E94172412BC11BC25
S1231D000E94E8000E9411010E949A000E946100809100019091010185FD07C080916F0044
S1231D208B7F80936F00449A449A8091260110928D0510921B0580911401909115018D5DE2
S1231D40954030F08CED95E090931501809314011092780586B3866086BB78948AEA0E949A
S1231D60C12280E00E94C12285E50E94C12289B1829586958695817080938A0580916E000F
S1231D80836080936E002B9A459A2C9AA89580917B0590917C058E37910570F180917805B7
S1231DA0882351F58091EC059091ED059F7E9093ED058093EC0580916F00856080936F00FC
S1231DC080916E00836080936E002B9A81E0809378058091EC059091ED0580629093ED055A
S1231DE08093EC058091EC059091ED0590629093ED058093EC0547C080917805813009F07C
S1231E0042C080917B0590917C058E379105D8F580916F008D7F80936F00809170008C7FC7
S1231E208093700080916F008B7F80936F0080916E00836080936E008091EC059091ED0517
S1231E408F7D9093ED058093EC058091EC059091ED05877F9093ED058093EC053898399884
S1231E603A983B9854985598449A449A109278058091EC059091ED059F7D9093ED058093AC
S1231E80EC0510927605809178058130F9F4809176058823C1F080916F00826080936F0038
S1231EA08091700083608093700080916E00836080936E008091EC059091ED058860909334
S1231EC0ED058093EC052B9A2C9A13C010927605449A449A109276051092B3001092820536
S1231EE01092810580913F0190914001892B09F42B9840917B0550917C0520912201309147
S1231F002301809100019091010180709074822B932B4817590788F48091EC059091ED05B5
S1231F2097FD0BC08091EC059091ED059F7B9093ED058093EC05469A0AC08091EC05909129
S1231F40ED0590649093ED058093EC054698F89480918305909184058A5A9A4AC1F0809147
S1231F608305909184058555954589F078948091EC059091ED0580649093ED058093EC05E0
S1231F8088EE93E090933501809334010AC078948091EC059091ED058F7B9093ED05809396
S1231FA0EC05F89480918505909186058A5A9A4AC1F080918505909186058555954589F06C
S1231FC078948091EC059091ED0580689093ED058093EC0588EE93E0909335018093340151
S1231FE00AC078948091EC059091ED058F779093ED058093EC0580913401909135010B9794
S123200058F02D9A80913401909135010197909335018093340101C02D9880911B0583306D
S123202009F4F7C0843018F4882371F08BC0853009F42BC2853008F456C1863009F4E3C113
S1232040873009F0DAC269C28091790590917A058D52914008F4D4C2E0911B05F0E0809122
S12320607800909179008C7F65E070E00E94A623EE0FFF1FE85AFA4F7183608380911B0591
S1232080C82FD0E0E0911B05F0E0EE0FFF1FE45EFA4F80819181E0911B05F0E0EE0FFF1FFF
S12320A0E85AFA4F20813181880F991F880F991F820F931F880F991F6AE070E00E94A62309
S12320C0CC0FDD1FC45EDA4F7983688310927A051092790580911B058F5F80931B0580914F
S12320E01B0580937C000E940B0880911C0590911D058A35910564F42091140130911501B9
S1232100C901880F991F820F931F9695879504C08091140190911501909317018093160192
S123212080913F0190914001892B09F464C280913F019091400101979093400180933F010F
S12321402B9A59C28091790590917A058D52914008F456C290911B0540918E05842F83705D
S12321608450990F990F980FE92FF0E0EE0FFF1FEE5FFE4F8081918120917800309179007D
S1232180820F931F969587959183808310927A0510927905A89580911B05C42FD0E0813097
S12321A071F48E01085F1F4F842F0E941E06000F111F045E1A4FF801918380830CC08081F2
S12321C0918162E070E00E94BA23CC0FDD1FCC5CDA4F7983688380911B058F5F80931B0577
S12321E080911B0580937C0080912C0590912D058D38910514F082E309C080912C05909196
S12322002D05893791050CF4FBC189E180937705F7C18091790590917A058D52914008F4EA
S1232220EFC1E0911B05F0E080917800909179009695879596958795EE0FFF1FE85AFA4F32
S12322409183808380911B05C82FD0E0E0911B05F0E0EE0FFF1FE45EFA4F80819181E09100
S12322601B05F0E0EE0FFF1FE85AFA4F20813181880F991F880F991F820F931F65E070E0FB
S12322800E94A623CC0FDD1FC45EDA4F7983688310927A051092790580911B058F5F809353
S12322A01B0580911B0580937C000E940B08A89580918E058F5F80938E05843010F01092BA
S12322C08E0590918E05292F27952227279585B18F77822B85B99295990F907485B18F7B60
S12322E0892B85B98DC18091790590917A058159914008F485C180912601882331F1E09108
S12323001B05F0E08091780090917900969587959695879590E0EE0FFF1FE85AFA4F9183EE
S12323208083A0911B05B0E0E0911B05F0E0EE0FFF1FE85AFA4F80819181AA0FBB1FA45E06
S1232340BA4F11969C938E933EC0E0911B05F0E08091780090917900EE0FFF1FE85AFA4F51
S12323609183808380911B05C82FD0E0E0911B05F0E0EE0FFF1FE45EFA4F00811181E091DF
S12323801B05F0E0EE0FFF1FE85AFA4F808191810E94DE069C01220F331F280F391FC80192
S12323A043E0880F991F4A95E1F7801B910B820F931F6AE070E00E94A623CC0FDD1FC45E78
S12323C0DA4F7983688310927A051092790580911B058F5F80931B0580911B0580937C0096
S12323E020918A0589B1829586958695817030E090E02817390709F4FEC0E0918F05F091E1
S123240090050995F8C08091790590917A058D52914008F4F5C0E0911B05F0E08091780053
S1232420909179009695879596958795EE0FFF1FE85AFA4F9183808380911B05C82FD0E0DB
S1232440E0911B05F0E0EE0FFF1FE45EFA4F80819181E0911B05F0E0EE0FFF1FE85AFA4F57
S123246020813181880F991F880F991F820F931F880F991F6AE070E00E94A623CC0FDD1FF9
S1232480C45EDA4F798368833EC08091790590917A058D52914008F4B3C0E0911B05F0E059
S12324A080917800909179009695879596958795EE0FFF1FE85AFA4F91838083E0911B0519
S12324C0F0E0EE0FFF1FE85AFA4F2081318184E190E0FC012E9FC0012F9F900D3E9F900DEA
S12324E011240E9484069093270580932605809126059091270562E070E00E94BA2370934D
S123250027056093260510927A051092790580911B058F5F80931B0568C080917905909102
S12325207A058D52914008F46BC0E0911B05F0E0809178009091790096958795969587952F
S123254090E0EE0FFF1FE85AFA4F918380838091660590916705893791050CF1A0911B059D
S1232560B0E0E0911B05F0E0EE0FFF1FE45EFA4F40815181E0911B05F0E0EE0FFF1FE85A6F
S1232580FA4F20813181CA01880F991F840F951F820F931F969587959695879519C0A0915F
S12325A01B05B0E0E0911B05F0E0EE0FFF1FE45EFA4F20813181E0911B05F0E0EE0FFF1F91
S12325C0E85AFA4F80819181820F931F96958795AA0FBB1FA45EBA4F11969C938E93109298
S12325E07A051092790510921B0580911B0580937C000E940B08A89503C081E080931B056D
S12326008091790590917A05019690937A058093790580917B0590917C058F55914008F4D9
S123262057C0809110068F5F809310069091100680911106981708F44EC010921006809160
S12326402A0590912B05E0911C06FF27E7FDF095E251FA4F208130E08217930734F480913B
S12326600E0690910F06890F17C080912A0590912B05E0911C06FF27E7FDF095E251FA4F6E
S1232680208130E0821793074CF080910E0682302CF080910E06815080930E0680910E06E1
S12326A0E0911C06FF27E7FDF095E251FA4F2089992787FD909530E02817390764F4E0910E
S12326C01C06FF27E7FDF095E251FA4F808901C081E080930E0680917B0590917C05873984
S12326E0910508F461C020912805309129058091240190E04996281739070CF055C0809130
S1232700B8059091B90501969093B9058093B8052091B8053091B9058091BA059091BB0533
S12327202817390708F442C01092B9051092B80520917B0530917C058091B2059091B30545
S12327402817390730F49091B6058091B705890F15C020917B0530917C058091B205909160
S1232760B30549968217930758F49091B6058091B505891728F48091B60581508093B60571
S12327809091B6058091B405891718F48091B40508C09091B6058091B505981738F48091BE
S12327A0B5058093B60502C01092B60580911A0582FF1BC080917B0590917C05805D9740FB
S12327C0A0F420912805309129058091240190E00596281739074CF481E080938C0580917E
S12327E0EC059091ED05916007C010928C058091EC059091ED059E7F9093ED058093EC059B
S1232800809100019091010192FF27C020917B0530917C0580912E0190912F0182179307D0
S1232820E0F420917B0530917C0580913001909131012817390788F42091280530912905F0
S12328408091240190E005962817390734F48091EC059091ED05946005C08091EC0590919B
S1232860ED059B7F9093ED058093EC05809100019091010193FF37C04A9935C020917B0568
S123288030917C0580913201909133018217930730F48091EC059091ED05986005C080911F
S12328A0EC059091ED05977F9093ED058093EC0580911A0583FF0DC080917B0590917C052F
S12328C0875D964030F08091BC059091BD05886005C08091BC059091BD05877F9093BD0518
S12328E08093BC0539C08091BC059091BD05877F9093BD058093BC058091370120912A056A
S123290030912B0590E082179307BCF040917B0550917C0520911E0130911F0180910001FD
S12329209091010180709078822B932B8417950750F480911A0580FF06C08091EC059091FA
S1232940ED05986005C08091EC059091ED05977F9093ED058093EC0580910001909101014B
S123296080FF48C080912D0180FF12C08091AF05883C28F08091B6058823C1F419C0909175
S1232980B6058091AF0586958917A8F0549813C080912D0182FF0FC08091AF05883C58F041
S12329A08091EC059091ED0596FF02C0549A01C054981092AF0580912D0184FF1DC0809106
S12329C0AF05883C50F080910E06181614F4559A01C055981092AF050FC020910E06809148
S12329E0AF05332727FD3095869590E0821793071CF001C0549855988091AF058F5F8093B2
S1232A00AF05C2C91F920F920FB60F9211248F939F9380911D068F5F80931D0680911D06A6
S1232A20882309F446C08091EC059091ED0590619093ED058093EC05109278058091EC05A4
S1232A409091ED059F7D9093ED058093EC0580916F008B7F80936F0080916F008D7F80937F
S1232A606F00809170008C7F8093700080916E00836080936E00449A449A8091EC05909112
S1232A80ED058F7D9093ED058093EC058091EC059091ED05877F9093ED058093EC05389817
S1232AA039983A983B985498559810927C0510927B0578949F918F910F900FBE0F901F9068
S1232AC018951F920F920FB60F9211248F9380912C01813019F482E08093C0058F910F9041
S1232AE00FBE0F901F9018958091AA05882309F466C02091AA058091AA05823089F4449A4F
S1232B008091850590918605880F991F9093860580938505809185059091860581600BC0DD
S1232B208091AA05803269F4449A8091850590918605880F991F9093860580938505109261
S1232B40AA0580918400909185009093B1058093B005479A8091E5059091E605892B61F0F9
S1232B6080911A06882341F08091E5059091E60590938B0080938A0080917B0590917C05BF
S1232B808C5D954008F04FC080911A0581FF4BC080918A0090918B0088539F4F90938B00F3
S1232BA080938A0020931A0680918A0090918B008C509E4F90931906809318060895809170
S1232BC01A06882381F120911A06223089F444988091830590918405880F991F90938405FA
S1232BE080938305809183059091840581600BC020911A06203269F4449880918305909131
S1232C008405880F991F90938405809383052093AA05809118069091190690938B008093FF
S1232C208A0010921A0608951F920F920FB60F9211242F933F934F935F936F937F938F931C
S1232C409F93AF93BF93EF93FF930E9474152B9A7894FF91EF91BF91AF919F918F917F919A
S1232C606F915F914F913F912F910F900FBE0F901F9018951F920F920FB60F9211242F93DA
S1232C808F939F93F8942091130120959091C005943001F1953040F4923019F19330A0F41E
S1232CA0913009F049C008C0973169F19336A9F19E3009F041C01BC02093B20084E0809381
S1232CC0B100389A83E042C026BD83E085BD3A9A84E03CC02093B2009093B1003B9A82E0DC
S1232CE035C026BD83E085BD399A81E02FC081E0809304052093B20084E08093B100389A54
S1232D003B9A87E123C081E08093050526BD83E085BD399A3A9A8EE019C081E0809304051E
S1232D202093B20084E08093B100389A3B9A3A9A399A9093C0050CC02093B20084E0809324
S1232D40B100389A3B9A3A9A399A83E68093C00578949F918F912F910F900FBE0F901F9059
S1232D601895CF93DF93EC0180918805E7E0F0E0E81BF109EE0FFF1FE45EFA4F80819181F6
S1232D8020918705821B282F30E080912B0190E0880F991F880F991FAC01429FC001439F72
S1232DA0900D529F900D112464E670E00E94A6236436710520F083E680931B0602C0609338
S1232DC01B0680911B066AE00E949A2380931406809114068A301CF089E08093140680912E
S1232DE07B0590917C058D5E9340C0F580917B0590917C0564E670E00E94A623655060935A
S1232E0017068091170618161CF01092170607C08091170685301CF085E080931706E091AE
S1232E201706FF27E7FDF095E65CFE4F808190E09093BF058093BE05109212068FEF8093DA
S1232E401C0680911406992787FD909534E0880F991F3A95E1F780937F05C7C080917B05FF
S1232E6090917C05875F9242E8F086E9809312068FE080931C068091140690911C06829557
S1232E80807F890F80937F05E0917F05F0E0EF5BFE4F808190E0880F991F9093BF058093EA
S1232EA0BE05A3C080917B0590917C05885E934062E370E00E94A6236093120680911206C8
S1232EC06AE00E949A2380931C068091140690911C068295807F890F80937F05E0917F0568
S1232EE0F0E0EF5BFE4F808190E0880F991F9093BF058093BE0580911C0687FD39C0809129
S1232F001C068F30ACF5E0917F05F0E0EE5BFE4F8081E0917F05F0E0EF5BFE4F6081E09121
S1232F20BE05F091BF052091120640911C06861B880F992787FD909530E06AE04602A001E5
S1232F401124241B350BAC01429FC001439F900D529F900D11246AE070E00E94BA23772771
S1232F6067FD70956E0F7F1F7093BF056093BE058091140687FD39C0809114068930ACF51F
S1232F80E0917F05F0E0EF5AFE4F8081E0917F05F0E0EF5BFE4F6081E091BE05F091BF051B
S1232FA020911B0640911406861B880F992787FD909530E06AE04602A0011124241B350BB8
S1232FC0AC01429FC001439F900D529F900D11246AE070E00E94BA23772767FD70956E0FBF
S1232FE07F1F7093BF056093BE0580917B0590917C05855F914010F45AEB69C080917B05C7
S123300090917C058952934210F05DE060C080917B0590917C0585569941B8F080917B05DC
S123302090917C05845699416AE070E00E94A623CB01880F991F880F991F860F971F64E632
S123304070E00E94A623562F42C080917B0590917C05815A9F40B8F080917B0590917C0562
S1233060805A9F406AE070E00E94A623CB01F3E0880F991FFA95E1F764E670E00E94A62334
S1233080562F545124C080917B0590917C05855F914010F450E01BC080917B0590917C05F4
S12330A0845F91406AE070E00E94A623CB019B01E3E0220F331FEA95E1F7880F991F820F6E
S12330C0931F64E670E00E94A623562F57532091BE053091BF05852F992787FD9095820F5F
S12330E0931F97FF06C08091BE059091BF0551E0581B40919405445645310CF044E1209115
S1233100BE053091BF05809112019091770520583040280F311D291B3109842F4C3E0CF47A
S12331208CEE682F772767FD7095620F731F852F992787FD9095680F791F42E06935740709
S12331402CF068E572E080E090E00CC0653071052CF465E070E080E090E004C0882777FD9D
S12331608095982F20917D0530917E052C0F3D1F40E050E00E947B2328E037E040E050E062
S12331800E94CD23C21BD30BCE01DF91CF910895CF93DF93EC016091AC057091AD052091DB
S12331A0130126952695620F711D7695679580E090E02AE530E040E050E00E947B2320914B
S12331C07D0530917E052C0F3D1FE3E036952795EA95E1F740E050E00E94CD23E0911C0678
S12331E0FF27E7FDF095EF50FB4FE08164EB70E06E1B7109882777FD8095982F620F731FAE
S1233200841F951F9E0140E050E00E947B2322E130E040E050E00E94CD23CA01B9012AE0A0
S123322030E040E050E00E94CD232A97CE01A0E0B0E02A9682179307A407B50718F48AE028
S123324090E003C0CE01821B930BDF91CF9108951F93CF93DF9380918400909185009093DC
S123326022068093210680918400909185008639910508F49FC280911D06882349F088EE6D
S12332809DEF909303058093020510921D065AC0E0918400F0918500C0910205D0910305BE
S12332A09E0136952795CE016AE070E00E94A623261B370BE217F30768F481E080932006A4
S12332C080912C01823009F075C28091F0048093C00570C280917B0590917C05E0917D0595
S12332E0F0917E0520918400309185008091EF0490E02C1B3D0BAC01429FC001439F900D7A
S1233300529F900D11246EE170E00E94BA23CB018E0F9F1F62E070E00E94BA2370937E050A
S123332060937D0510927E0510927D05809184009091850090930305809302051092850024
S12333401092840080917605893628F4809176058F5F8093760580917B0590917C058052CF
S1233360934040F4449B02C0449904C0449A449A1092AA05479880917B0590917C05C09190
S12333800205D0910305D093EB05C093EA052091EA053091EB051091810040E050E060E021
S12333A070E489E191E00E94EF23CA01B9012EE130E040E050E00E947B2320EC129F9001A4
S12333C0112420503240442737FD4095542F0E94CD2330937C0520937B052091A1053091BA
S12333E0A20540919F055091A005C901880F991F820F931F840F951F9695879596958795F6
S12334009093A2058093A10580919D0590919E059093A00580939F0580919B0590919C05BC
S123342090939E0580939D058091990590919A0590939C0580939B058091970590919805BC
S123344090939A05809399058091950590919605909398058093970580917B0590917C05EC
S1233460909396058093950580917B0590917C058D5D9540D8F040919405809195059091ED
S123348096052091A1053091A205821B930B23E0429FA0011124840F951F24E09695879547
S12334A02A95E1F78B5A809394050FC084E68093940580917D0590917E0564E070E00E948E
S12334C0BA2370937E0560937D0510921D0680917B0590917C058C52914000F580918100E2
S12334E08330E1F4809120068823C1F484E0809381001092850010928400D695C795D69532
S1233500C795D0930305C09302058091EA059091EB05969587959695879526C080917B0570
S123352090917C058D5B924018F1809181008430F9F4809120068823D9F483E08093810049
S12335401092850010928400CC0FDD1FCC0FDD1FD0930305C09302058091EA059091EB0596
S1233560880F991F880F991F9093EB058093EA058091EA059091EB050E94B11690931906D8
S12335808093180680917B0590917C058A58924018F484E690E009C080917B0590917C052D
S12335A08E57944038F482E390E090931F0680931E0604C010921F0610921E06809118064E
S12335C090911906209116013091170140911E0650911F06821B930B841B950B9093160652
S12335E080931506809115069091160697FF20C080911506909116062091EA053091EB0500
S12336004091180650911906820F931F8417950778F42091EA053091EB0580911806909130
S12336201906821B930B44969093160680931506F89480917B0590917C05805E9E4208F070
S12336408EC08091EC059091ED0593FD88C080911506909116068536910504F11092AA052B
S1233660809115069091160690938B0080938A0080918A0090918B009093E6058093E50540
S123368080912006882311F480E201C082E080931A061092AA0584E090E055C08091150621
S12336A0909116068B5B9F4F14F11092AA0584E690E090938B0080938A009093E605809359
S12336C0E50580912006882311F480E201C082E080931A0644981092AA0588E290E0909333
S12336E0E8058093E70584E18093010530C0809118069091190690938B0080938A00209101
S1233700EA053091EB058091150690911606820F931F9093E6058093E5058091200688236C
S123372031F4449880E28093AA0582E005C0449882E08093AA0580E280931A0684E180932C
S1233740010584EB90E09093E8058093E705109220068091EC059091ED059F770FC080919E
S1233760EA059091EB058C509E4F90938B0080938A008091EC059091ED0590689093ED050F
S12337808093EC0580917B0590917C058D5A9D4038F080918400909185008C599F4F06C02E
S12337A08091EA059091EB050E94C81890938900809388007894DF91CF911F9108951F9251
S12337C00F920FB60F9211242F933F934F935F936F937F938F939F93AF93BF93EF93FF9331
S12337E00E9428192B9A7894FF91EF91BF91AF919F918F917F916F915F914F913F912F91B1
S12338000F900FBE0F901F9018951092800081EF9FEF909389008093880085EF9FEF9093B1
S12338208B0080938A0080E880938100109285001092840084E08093810080916F008760B4
S123384080936F00539852983C9A3D9A449A449AA2E0B2E00E940A24802D8093EF04A1E08C
S1233860B2E00E940A24802D8093F0048091F0048E3039F08091F004873119F087E1809301
S1233880F00480918905813021F4809169008C6003C080916900886080936900E99A0895A4
S12338A021EB30E0F90110821092B6001092B2001092B300A0E7B0E08C9183608C93389855
S12338C04098399841983A9842983B984398389839983A983B98EFE6F0E080818D7F80830D
S12338E08C918C7F8C9386E0F901808384E68093E1050895813099F438983B9880912C01FB
S1233900843021F439983A98109205051092260610922506109204051092B10008958230A3
S123392049F439983A9810922406109223061092050515BC08951F920F920FB60F92112405
S12339402F933F934F935F936F937F938F939F93AF93BF93EF93FF93F89480910405843091
S123396019F481E00E947A1C7894FF91EF91BF91AF919F918F917F916F915F914F913F91F1
S12339802F910F900FBE0F901F9018950F931F9380911C0590911D050A9714F487E003C060
S12339A080918C0586E08093B1001092B20080917B0590917C05845F914018F41092170631
S12339C016C080917B0590917C058D56974020F08EE0809317060BC080917B0590917C0574
S12339E064E670E00E94A623655060931706E0911706F0E0E55DFC4F8081809313018091D5
S1233A008C05882329F02091F1018091180108C0E0917F05F0E0EF51FE4F8081209118019B
S1233A20829FC00111249093AD058093AC0580917B0590917C05825C914048F580910001A1
S1233A409091010182FF19C08091AC059091AD0520911901820F911D9093AD058093AC05AD
S1233A608091EC059091ED0584609093ED058093EC058EE18093AB053FC08091EC059091DC
S1233A80ED058B7F9093ED058093EC0535C08091EC059091ED058B7F9093ED058093EC05E0
S1233AA08091AB05823028F08091AB0581508093AB05E091AC05F091AD05809119012091F1
S1233AC019014091AB05E80FF11D8EE190E0841B910930E0AC01429FC001439F900D529F5B
S1233AE0900D11246EE170E00E94A623E61BF70BF093AD05E093AC0580918C05882309F044
S1233B00ABC1E0917F05F0E0EF51FE4F808120911801829FC00111249093AD058093AC0568
S1233B2080911C0687FD3EC080911C068F30D4F5E0917F05F0E0EE51FE4F6081E0917F05EA
S1233B40F0E0EF51FE4F40810091AC051091AD058091120620911C06E091180170E0641B59
S1233B60710990E04AE0240290011124821B930B9C01629FC001639F900D729F900D112425
S1233B806AE070E00E94BA23F0E06E9FC0016F9F900D7E9F900D1124800F911F9093AD05BC
S1233BA08093AC058091140687FD3EC0809114068930D4F5E0917F05F0E0EF50FE4F6081B1
S1233BC0E0917F05F0E0EF51FE4F40810091AC051091AD0580911B0620911406E0911801B2
S1233BE070E0641B710990E04AE0240290011124821B930BAC01649FC001659F900D749F92
S1233C00900D11246AE070E00E94BA23F0E06E9FC0016F9F900D7E9F900D1124800F911F3E
S1233C209093AD058093AC05809100019091010184FF55C0209146053091470580912805D3
S1233C409091290528173907C4F480912805909129052091460530914705821B930B64E0C5
S1233C6070E00E94BA2380918005861710F460938005809125018093AE053091AE053430ED
S1233C80C8F08091AC059091AD05E0918005F0E0EF5DFC4F2081820F911D9093AD058093AE
S1233CA0AC0531503093AE058091EC059091ED05806109C0109280051092AE058091EC051B
S1233CC09091ED058F7E9093ED058093EC058091280590912905909347058093460580913C
S1233CE000019091010191FFB4C080918A05882309F0AFC08091E3058F5F8093E3059091E2
S1233D00E3058091E405981708F4A6C01092E3058091240590912505E0911406FF27E7FD08
S1233D20F095EF53FA4F208130E028173907B4F48091240590912505E0911406FF27E7FD7D
S1233D40F095EF53FA4F2081821B910962E070E00E94BA236C596093E1052BC080912405A3
S1233D6090912505E0911406FF27E7FDF095EF53FA4F208130E082179307DCF48091E105A4
S1233D801816BCF4E0911406FF27E7FDF095EF53FA4F8081209124053091250590E0821BC9
S1233DA0930B62E070E00E94BA2384E6861B8093E1058091EC059091ED059D7F9093ED0506
S1233DC08093EC052091E105E0911406FF27E7FDF095EF53FA4F8089332727FD309590E0E3
S1233DE08C599F4F8217930754F4E0911406FF27E7FDF095EF53FA4F80898C591EC020914F
S1233E00E105E0911406FF27E7FDF095EF53FA4F4089332727FD309584E690E0841B9109F4
S1233E2028173907CCF4E0911406FF27E7FDF095EF53FA4F908984E6891B8093E105809169
S1233E40EC059091ED0592609093ED058093EC0503C084E68093E105209132053091330548
S1233E6080911B0190E0C296281739070CF042C0809100019091010181FF3CC080913205D3
S1233E8090913305C397D4F040911A0180911A01209132053091330560911B0190E070E0E1
S1233EA06E5C7F4FFC01E29FC001E39F900DF29F900D11240E94A623461B03C080911A01EA
S1233EC0482F50E08091AC059091AD05480F591F5093AD054093AC05809120019091210145
S1233EE090931F0180931E018091EC059091ED0582600DC080911C0190911D0190931F01D5
S1233F0080931E018091EC059091ED058D7F9093ED058093EC0580912601882371F020913C
S1233F20AC053091AD058091E10524563040992787FD9095280F391F0DC02091AC05309190
S1233F40AD058091E1052C593F4F992787FD9095281B390B3093AD052093AC058091BC0506
S1233F609091BD0583FF1CC0E091AC05F091AD05209139018091AC059091AD0564E170E092
S1233F800E94BA2330E0629FC001639F900D729F900D11248E0F9F1F9093AD058093AC0556
S1233FA0809100019091010190FF4CC080911C0590911D05823891050CF044C08091AC05A6
S1233FC09091AD0520912701820F911D9093AD058093AC05E0911C05F0911D05609118011A
S1233FE02091270182E890E08E1B9F0B70E0AB01849FB001859F700D949F700D11248FEFE3
S123400090E0FB01E89FB001E99F700DF89F700D1124882777FD8095982F30E040E050E04B
S12340200E947B2320E43FE140E050E00E94CD238091AC059091AD05820F931F9093AD0589
S12340408093AC052091AC053091AD058091180145EF849FC00111248217930754F48091C0
S12340601801849FC00111249093AD058093AC050BC08091AC059091AD051816190624F0B0
S12340801092AD051092AC0520918105309182058091AC059091AD05820F931F96958795D7
S12340A0909382058093810540917B0550917C0520911E0130911F01809100019091010120
S12340C080709078822B932B4817590730F48091EC059091ED059F770DC080911A0580FDF1
S12340E004C0389839983A983B988091EC059091ED0590689093ED058093EC058091EC058A
S12341009091ED0592FF04C0389839983A983B9878941F910F9108951F920F920FB60F923C
S123412011242F933F934F935F936F937F938F939F93AF93BF93EF93FF93F8942091040588
S1234140223039F0243009F44FC0213009F051C01CC080912506909126068F3F9105D1F19A
S1234160C8F180912506909126068F5F8093B30080912506909126068F5F904090932606AF
S1234180809325062093040534C00E94C61C809181059091820590932606809325068091CC
S12341A02506909126068F3F9105A1F098F080912506909126068F5F8093B300809125068D
S12341C0909126068F5F9040909326068093250682E007C080912506909126068093B300CB
S12341E084E08093040505C081E00E947A1C109204057894FF91EF91BF91AF919F918F9136
S12342007F916F915F914F913F912F910F900FBE0F901F9018951F920F920FB60F921124D6
S12342202F933F934F935F936F937F938F939F93AF93BF93EF93FF93F89480912C01843084
S123424008F05EC020910505223039F0243009F453C0213009F082C020C0809123069091E3
S123426024068F3F910591F088F080912306909124068F5F87BD80912306909124068F5F89
S12342809040909324068093230633C0809123069091240687BD84E024C080918105909105
S12342A08205909324068093230624E025BD16BC80912306909124068F3F9105A9F0A0F020
S12342C080912306909124068F5F87BD80912306909124068F5F9040909324068093230657
S12342E082E0809305053AC0809123069091240687BD2093050532C082E00E947A1C2EC041
S123430080912D0181FD04C080912D0185FF23C084E085BDE0917F05F0E0EF57FD4F808174
S12343208C5E87BD8091EC059091ED0597FD16C08091EC059091ED0592FD10C087B58F315C
S123434068F080912D0181FD549A80912D0185FF05C0559A03C016BC81E087BD7894FF9109
S1234360EF91BF91AF919F918F917F916F915F914F913F912F910F900FBE0F901F90189502
S12343801F920F920FB60F9211242F933F934F935F936F937F938F939F93AF93BF93EF9346
S12343A0FF93F89480912C01843040F480910505843061F482E00E947A1C08C080912D01F0
S12343C081FD549880912D0185FD55987894FF91EF91BF91AF919F918F917F916F915F91C5
S12343E04F913F912F910F900FBE0F901F90189554985C9855985D985498559815BCEEE6A2
S1234400F0E080818360808384E085BD16BC82E187BD089511B88FEF84B915B887B98AB951
S12344200895089508950895089588E98093C10083E18093C4008EE696E090932C06809395
S12344402B0690932806809327068EE296E090932A06809329069093AF068093AE061092DA
S12344602D061092E90508951F920F920FB60F9211248F939F93EF93FF9380912D06882394
S123448011F1E0912B06F0912C0681918093C600F0932C06E0932B06EE5AF64030F08EE66B
S12344A096E090932C0680932B0680912D06815080932D0680912D06882329F48091C100B0
S12344C08F7D8093C100FF91EF919F918F910F900FBE0F901F9018951F920F920FB60F9279
S12344E011242F938F939F93EF93FF938091C600E091AE06F091AF0680838091E9058F5F37
S12345008093E9058091AE069091AF0601969093AF068093AE068E56964030F08EE296E005
S12345209093AF068093AE06FF91EF919F918F912F910F900FBE0F901F9018958091E90552
S1234540882319F48FEF9FEF0895F8948091E90581508093E905E0912906F0912A06219196
S1234560F0932A06E0932906EE56F64030F08EE296E090932A06809329067894822F90E0A0
S12345800895982F80912D068F33E0F780912D06803418F080E090E00895F89480912D0699
S12345A08F5F80932D06E0912706F0912806908380912706909128060196909328068093DB
S12345C027068E5A964030F08EE696E090932806809327068091C10080628093C1007894BD
S12345E081E090E00895CF93DF93EC0104C00E94C1228111219688818823C9F781E090E0B1
S1234600DF91CF91089586E095E00E94F32208958EE095E00E94F32208958091E90590E054
S12346200895CF92DF92EF92FF920F931F93CF93DF93CDB7DEB729970FB6F894DEBF0FBE39
S1234640CDBF8C01F62EE42EDE011196E1E1F5E089E001900D928150E1F749E06E01089474
S1234660C11CD11CFF2081F089E090E0841B91092F2D30E08217930738F04150F601E40F88
S1234680F11D8CE28083FF244150F601E40FF11DC8016AE070E00E94A623805D8083C80174
S12346A06AE070E00E94A6238B01672B11F4FF2019F085E08F15B0F619E01E197E010894AC
S12346C0E11CF11C07C0F701E10FF11D80810E94C1221F5F1930B8F329960FB6F894DEBF6A
S12346E00FBECDBFDF91CF911F910F91FF90EF90DF90CF900895629FD001739FF001829FCE
S1234700E00DF11D649FE00DF11D929FF00D839FF00D749FF00D659FF00D9927729FB00DB0
S1234720E11DF91F639FB00DE11DF91FBD01CF0111240895991B79E004C0991F961708F0FC
S1234740961B881F7A95C9F780950895AA1BBB1B51E107C0AA1FBB1FA617B70710F0A61B09
S1234760B70B881F991F5A95A9F780959095BC01CD01089597FB092E07260AD077FD04D00B
S1234780E5DF06D000201AF4709561957F4F0895F6F7909581959F4F0895A1E21A2EAA1BA4
S12347A0BB1BFD010DC0AA1FBB1FEE1FFF1FA217B307E407F50720F0A21BB30BE40BF50BB2
S12347C0661F771F881F991F1A9469F760957095809590959B01AC01BD01CF01089597FB13
S12347E0092E05260ED057FD04D0D7DF0AD0001C38F450954095309521953F4F4F4F5F4F66
S12348000895F6F790958095709561957F4F8F4F9F4F0895F999FECFB2BDA1BDF89A119639
S123482000B40895F7DFE02DF5DFF02D0895F999FECFB2BDA1BD00BC11960FB6F894FA9A3E
S1234840F99A0FBE0895F3DF012CF1DF11240895FFCF2F00010002000300040005000600A4
S1234860070008003228E803900106141E3C581B581B88136419121E01010203040A041183
S1234880C4098813AC0D6400DCE603020A14324696500054819596B7AFC3C8BEBEB9B0AFC7
S12348A0AFADAC4984C0CBD2D6D7D0C7C2BBB8B3AEAAA9458AA2A9AAB7C0BABEBBB6B8B207
S12348C0B3B4B93281868DA4A58B8C8F9EA6A2A6A5A6C034525D5B596F788285858281FF5C
S12348E0859FB034444E4B4A54615769727272737D9095272C1B252B334B5155616A6D6C1F
S12349007D828B1D211A242A32454C4F5E6169717E818634323232323232323232327F325A
S123492032323232323232323232323232323232323232131718191B1C1D1F212325272837
S12349402C2E311418191A1C2124272B3035393C3E414316191D232A31353B3F42484E5673
S12349605A5E651B1D363E525863666C6E777D84898D932226434B6172818A9097A8ACAF1E
S1234980B1B6B9292E484E6B7C939BA2AFB9BFCBD2D2D229344B536E7F9CA8B1BCC5D0D2E7
S12349A0D2D2D2283F4E587187A4B2BAC2D2D2D2D2D2D23746545E7691B1BEC4D2D2D2D209
S12349C0D2D2D239485660869FBAD2D2D2D2D2D2D2D2D200000000000000000000000000E5
S12349E00000000000000000000000000000000000000000000000000000000000000000B3
S1234A00000000000000000000000000000000000000000102030405060708090A0B0C0D37
S1234A200E0F100102030405060708090A0B0C0D0E0F100102030405060708090A0B0C0D62
S1234A400E0F1014161718191A1B1C1D1E1F2021222324191A1B1C1D1E1F202122232425CB
S1234A602627271E1F2022232425262728292A2B2C2D2E000204060708090A0C0E2826249F
S1234A8022201E1E1E1E1E1E1E1E1E1E1EF0FF80BBE0880465484BA438022BF0207019CC8A
S1234AA013860F440CC209D0074C061B052A046A03D1025602F201A1015F012801FB00D631
S1234AC000B7009D0087007500660059004D0044003C0034002E0029002500F0FF80BBE03C
S1234AE0880465484BA438022BF0207019CC13860F440CC209D0074C061B052A046A03D148
S1234B00025602F201A1015F012801FB00D600B7009D0087007500660059004D0044003C6C
S1234B200034002E0029002500F0FF80BBE0880465484BA438022BF0207019CC13860F44D9
S1234B400CC209D0074C061B052A046A03D1025602F201A1015F012801FB00D600B7009D28
S1234B600087007500660059004D0044003C0034002E0029002500F0FF80BBE088046548B6
S1234B804BA438022BF0207019CC13860F440CC209D0074C061B052A046A03D1025602F294
S1234BA001A1015F012801FB00D600B7009D0087007500660059004D0044003C0034002EB6
S1234BC000290025000000F5047E05AE066C08C00AB30D630F8B10D7118813000000000ABB
S1234BE0000F001E003C007800FA007201E00180028002000008000A000C000E00C80A4A36
S1234C00067E0484031A002000270032003E0066008E00B202EB02240337034B03560361B2
S1234C20037003E800D600C200B0009D008A00780078006500520040002D0019000700006F
S1234C400001175A5A5A505050505050505050505050503200FA04041B5B481B5B324A0036
S10F4C600D0A002020202020202020200D
S503026496
